:020000040000FA
:040000002BEF03F0EF
:08000800E8CF05F0D8CF06F0A7
:10001000E0CF07F00001E9CF0DF0EACF08F0E1CF23
:1000200009F0E2CF0AF0D9CF0BF0DACF0CF0F3CF22
:1000300014F0F4CF15F0FACF16F000C00FF001C0A5
:1000400010F002C011F003C012F004C013F09DAA1A
:100050002DEF00F09EBABCEF00F00FC000F010C012
:1000600001F011C002F012C003F013C004F00DC083
:10007000E9FF08C0EAFF09C0E1FF0AC0E2FF0BC0C8
:10008000D9FF0CC0DAFF14C0F3FF15C0F4FF16C08F
:10009000FAFF05C0E8FF07C0E0FF06C0D8FF100068
:1000A000F2CF0EF0F29EF76ABA0FF66E000EF7224C
:1000B0000900F5500EBEF28E12004F4B0A0D0000E3
:1000C000F2CF0EF0F29EF76ADA0FF66E000EF7220C
:1000D0000900F5500EBEF28E1200256C750A0D4D0A
:1000E0004158313434204348303A20256C752C2057
:1000F00025662C20256C750A0D00F2CF0EF0F29EBD
:10010000F76A140FF66E010EF7220900F5500EBEC5
:10011000F28E12004D4158313434204348313A2098
:10012000256C752C2025662C20256C750A0D000089
:10013000F2CF0EF0F29EF76A4A0FF66E010EF7222A
:100140000900F5500EBEF28E12004144433A2025BC
:100150006C752C2025662C20256C750A0D0A0D0067
:100160009EAAFED7ABCF18F0AECF01F018A202D0F6
:10017000AB98AB880000000CF3DF01C03FF4040132
:100180003F51120A000101E02DD0EADF015034088E
:1001900002E0000E01D0010E0401426F0001E0DF19
:1001A0000150560802E0000E01D0010E0401421574
:1001B000446F0001D5DF0150780802E0000E01D045
:1001C000010E04014415466F0001CADF015090087A
:1001D00002E0000E01D0010E04014615D8A4FF0074
:1001E000000100D09E9A2DEF00F0040EEA6E250E5D
:1001F000E96EEF500EE00F0E016E006A002EFED782
:10020000012EFBD78F0E006E002EFED70000EF2EC2
:10021000F2D7000C8E0E006E25C401F024C402F04B
:10022000036A015209E102C001F0026A080E005E91
:10023000015202E1006A08D0D89001BE04D0023613
:1002400001360006F9D7019E0000000C040132516E
:10025000D8B471D0006E3651D8B46DD0002604E306
:10026000810E002668E204D07F0E005E64E363E046
:1002700033C43AF437513A1B338F378F3551390332
:10028000F4CF3CF434513803F4CF03F0F3CF3BF414
:100290003903F3503C27F4503B23000E0322355121
:1002A0003803F3503C27F4503B23000E026A03222C
:1002B000022233513903F3503B27F4500322000E3E
:1002C000022233513803F3500326F4500222000E69
:1002D000016A012235513703F3503B27F4500322C2
:1002E000000E0222012234513703F3500326F4504A
:1002F0000222000E012233513703F3500226F4503C
:100300000122002A01BE05D03B37033602360136F2
:100310000006000E3BAF0AD0032A02220122015040
:1003200005E1025003E1035001E1002A3ABF018ECA
:100330003AAF019E04D0006A016A026A036A0000B3
:100340000001000CEACF2DF4E9CF2CF4040126398A
:10035000F009286F2827E20F296F320F2B6F2651E3
:100360000F0B292729272B27E90F2A6F2A272A274E
:1003700025390F0B2A272B272A372B372B1F2B37F3
:1003800025510F0B2B272837070E276F0A0E2A0738
:100390002B27FDE329072A27FDE328072927FDE36B
:1003A00027072827FDE3040EEA6E270EE96E070EE5
:1003B0002C152C9DE9262B0EE95CD8B42C8DEF5022
:1003C000006E08E12CBD06D02CB90CD02CB702D0A1
:1003D000200E03D02C872C99300E002600509EA8AA
:1003E000FED7AD6EEE502CADE6D70001000C040137
:1003F0003251B608326F036A33C436F4338FD89063
:100400003333343335330332023201320032322F88
:10041000F6D736AF0BD0001E011E021E031E002AA7
:10042000D8B4012AD8B4022AD8B4032A000185EF2F
:1004300002F0006A016A026A036A04013A6B3B6BCC
:100440003C6B3D6B39513811371136112CE0200EC1
:100450003E6FD89032373337343735373A373B37FA
:100460003C373D3739513D5D08E138513C5D05E190
:1004700037513B5D02E136513A5D0FE336513A5F49
:100480003751D8A0373D3B5F3851D8A0383D3C5F4D
:100490003951D8A0393D3D5FD8800036013602364B
:1004A00003363E2FD6D70000040EEA6E3A0EE96EF0
:1004B0000001000CE95004012A6F29512C6F1BE048
:1004C00028C435F427C434F426C433F425C432F4E4
:1004D000396B386B200E376F820E366F0001B6DE37
:1004E00003C028F402C027F401C026F400C025F49C
:1004F00004012C2FE5D728C435F427C434F426C4CE
:1005000033F425C432F4000172D703C028F402C0CA
:1005100027F401C026F400C025F4040128AF0DD053
:100520002A072A8B251F261F271F281F252BD8B4F3
:10053000262BD8B4272BD8B4282B3B0E316F9A0E1C
:10054000306FCA0E2F6F2E6B0A0E2C6F2951D8B444
:100550002A2B28C435F427C434F426C433F425C424
:1005600032F431C439F430C438F42FC437F42EC413
:1005700036F400015EDF0150EFCF25F4ECCF26F416
:10058000ECCF27F4ECCF28F4005213E10401292921
:100590002C5DD8A402D000010CD02A510DE00F0B25
:1005A0002C5D01E03CE22ABF3AD02ABD05D0200EE6
:1005B00031D0200E04012A172AAB0DD02A9B2951D5
:1005C000D8A42A0700502A6F2D0E9EA8FED7AD6E24
:1005D0002A51006E2A6B29512C5D0BE100502A6FC5
:1005E0002E0E9EA8FED7AD6E2A51006E200E2A1741
:1005F000000E300E2AAB0ED02A9B2951D8A42A0710
:1006000000502A6F2D0E9EA8FED7AD6E2A51006EA7
:100610002A6B300E002600509EA8FED7AD6E31C466
:1006200035F430C434F42FC433F42EC432F4396BAF
:10063000386B376B0A0E366F0001FBDE03C031F4F6
:1006400002C030F401C02FF400C02EF404012C2F9E
:1006500080D70001000CF86AD09E0D8EEA6AE96A24
:10066000B896190EAF6E260EAC6E900EAB6EC150E2
:10067000C00B0F09C16E070EB46E186AC150C00BD3
:100680000E09C16EC090C082C084C08EC280880E28
:10069000D56ECD6A000ECA6E7F0ECB6EB150480B80
:1006A0008509B16EB70EB1169484BD6ABD6AB116E4
:1006B0009482BA6ABA6A9D8AC00EF21293948A84AE
:1006C00093928A92000E016EC250C30B0110C26E4B
:1006D000010E0401256F000188DD1F6A1E6A020EEB
:1006E0000401246FFA0E256F00017FDD0401242F21
:1006F000F9D7246B24510001D3DC0401242B006EB4
:1007000000509EA8FED7AD6E040E245DF3E1C80E26
:10071000256F00016ADDB36AB26A0401246B939409
:100720008A94938081A0FDD7296B295107080FE394
:1007300093928A82D89028352A6F9380000E81B0D8
:10074000010E2A11286F93928A92292BEED728C482
:1007500001F001C027F4296B295107080FE3939298
:100760008A82D89028352A6F9380000E81B0010EBE
:100770002A11286F93928A92292BEED728C401F070
:1007800027C426F401C025F4000E26B9010E245D0D
:1007900038E093948A84000093948A94938081A093
:1007A000FDD7296B295107080FE393928A82D890CD
:1007B00028352A6F9380000E81B0010E2A11286F10
:1007C00093928A92292BEED728C401F001C027F416
:1007D000296B295107080FE393928A82D890283514
:1007E0002A6F9380000E81B0010E2A11286F939218
:1007F0008A92292BEED728C401F027C426F401C021
:1008000025F493948A842535276F2635286F27375A
:1008100028372737283727372837F00E271728316A
:10082000266F2731256F263325332633253326338C
:1008300025330F0E261725C401F026C402F002C08E
:100840001BF001C01AF0D8901E34026E1F34036EE4
:100850000250240FE96E000E0320EA6E1BC0ECFF6D
:10086000ED521AC0EFFFB250B3CF03F01C6E03C0BD
:100870001DF0236A226A200E216E750E206E1BC0A9
:1008800025F41AC024F40001C5DC03C035F402C00D
:1008900034F401C033F400C032F423C039F422C070
:1008A00038F421C037F420C036F4D0DC03C023F084
:1008B00002C022F001C021F000C020F0100EE96E4D
:1008C0001FC026F41EC025F43DDD030E0401246F75
:1008D0002451000160EC00F00401242B006E005054
:1008E0009EA8FED7AD6E110E245DF2E1100EE96EEA
:1008F0001BC026F41AC025F4000124DD2C0E9EA88E
:10090000FED7AD6E200E9EA8FED7AD6E890EE96EA5
:1009100023C028F422C027F421C026F420C025F4E7
:10092000060E0401296F0001C5DD2C0E9EA8FED71E
:10093000AD6E200E9EA8FED7AD6E100EE96E1DC0E6
:1009400026F41CC025F4FEDC0A0E9EA8FED7AD6E70
:100950000D0E9EA8FED7AD6EB36AB26A010E0401F9
:10096000246F93948A94938081A0FDD7296B295199
:1009700007080FE393928A82D89028352A6F9380D4
:10098000000E81B0010E2A11286F93928A92292BB2
:10099000EED728C401F001C027F4296B29510708BC
:1009A0000FE393928A82D89028352A6F9380000EA5
:1009B00081B0010E2A11286F93928A92292BEED7CB
:1009C00028C401F027C426F401C025F4000E26B97E
:1009D000010E245D38E093948A84000093948A94F5
:1009E000938081A0FDD7296B295107080FE39392CB
:1009F0008A82D89028352A6F9380000E81B0010E2C
:100A00002A11286F93928A92292BEED728C401F0DD
:100A100001C027F4296B295107080FE393928A82BA
:100A2000D89028352A6F9380000E81B0010E2A11CC
:100A3000286F93928A92292BEED728C401F027C4FD
:100A400026F401C025F493948A842535276F263532
:100A5000286F273728372737283727372837F00ECA
:100A600027172831266F2731256F26332533263364
:100A70002533263325330F0E261725C401F026C44F
:100A800002F002C01BF001C01AF0D8901E34026EB2
:100A90001F34036E0250240FE96E000E0320EA6E2D
:100AA0001BC0ECFFED521AC0EFFFB250B3CF03F002
:100AB0001C6E03C01DF0236A226A200E216E750E83
:100AC000206E1BC025F41AC024F400010AEC01F0CA
:100AD00003C035F402C034F401C033F400C032F472
:100AE00023C039F422C038F421C037F420C036F4D2
:100AF00026EC01F003C023F002C022F001C021F077
:100B000000C020F00401246B245100017DEC00F0B2
:100B10000401242B006E00509EA8FED7AD6E0C0E73
:100B2000245DF2E1100EE96E1BC026F41AC025F414
:100B3000000108DC2C0E9EA8FED7AD6E200E9EA8EC
:100B4000FED7AD6E890EE96E23C028F422C027F4CB
:100B500021C026F420C025F4060E0401296F0001EF
:100B6000A9DC2C0E9EA8FED7AD6E200E9EA8FED747
:100B7000AD6E100EE96E1DC026F41CC025F4A2EC6B
:100B800001F00A0E9EA8FED7AD6E0D0E9EA8FED7F0
:100B9000AD6EB36AB26AC282C2B2FED7C3CF1AF0D8
:100BA000C4CF1BF0D8901E34026E1F34036E025067
:100BB000240FE96E000E0320EA6E1BC0ECFFED521D
:100BC0001AC0EFFFB250B3CF03F01C6E03C01DF08C
:100BD000236A226A200E216E770E206E1BC025F438
:100BE0001AC024F40AEC01F003C035F402C034F456
:100BF00001C033F400C032F423C039F422C038F409
:100C000021C037F420C036F426EC01F003C023F0F5
:100C100002C022F001C021F000C020F00401246BCA
:100C20002451000198EC00F00401242B006E0050C8
:100C30009EA8FED7AD6E050E245DF2E1100EE96EA2
:100C40001BC026F41AC025F40001A2EC01F02C0E02
:100C50009EA8FED7AD6E200E9EA8FED7AD6E890E63
:100C6000E96E23C028F422C027F421C026F420C056
:100C700025F4060E0401296F00011CDC2C0E9EA831
:100C8000FED7AD6E200E9EA8FED7AD6E100EE96E9B
:100C90001DC026F41CC025F4A2EC01F0110E0401C5
:100CA000256F2551000198EC00F00401252B006E02
:100CB00000509EA8FED7AD6E150E255DF2E11E2AEE
:100CC000D8B41F2A1F50010802E21F6A1E6A040ED0
:100CD000246FFA0E256F0001F5EC00F00401242FBB
:080CE000F8D7000118D503004C
:020000040030CA
:0E000000240E3F1E008381000FC00FE00F4052
:00000001FF
